:100000000C94FA000C9419010C9419010C94190128
:100010000C9419010C94EB030C9419010C94190124
:100020000C9419010C9419010C9419010C941901E8
:100030000C94BF190C9419010C9419010C9419011A
:100040000C9419010C94C4030C94E61F0C94190130
:100050000C9419010C941B010C9419010C941901B6
:100060000C9419010C9419010C9419010C941901A8
:100070000C9419010C9419010C9419010C94190198
:100080000C9419010C9419010C9419010C94190188
:100090000C941901061008100A100C100E10101004
:1000A00012101410161018101A101C101E10201008
:1000B00022102410261028102A1054105410541006
:1000C0005410541054102C102E10301032103410C4
:1000D0003A103810361038103A103C103E104010CC
:1000E00042104410461048104A104E109D109F10A8
:1000F000A110A310A510A710A910AB10AD10AF1040
:10010000B110B310B510B710B910BB10BD10BF10AF
:10011000C110EB10EB10EB10EB10EB10EB10C31059
:10012000C510C710C910CB10D110CF10CD10CF10F3
:10013000D110D310D510D710D910DB10DD10DF107F
:10014000E110E51056115C11621168116E11741105
:100150007A11801186118C11921198119E11A4119F
:10016000AA11B011B611BC11C21153115311531180
:10017000531153115311C811CE11D411DA11E011DA
:10018000F211EC11E611EC11F211F811FE1104124A
:1001900010120A120A12101216121C12651268129C
:1001A0006B126E127112741277127A127D12801213
:1001B0008312861289128C128F1292129512981243
:1001C0009B126212621262126212621262129E121A
:1001D000A112A412A712AA12B312B012AD12B01239
:1001E000B312B612B912BC12C212BF12BF12C2129F
:1001F000C512C81211241FBECFEFD0E1DEBFCDBFA4
:1002000013E0A0E0B1E0E8E7F4E400E00BBF02C0D7
:1002100007900D92A633B107D9F716E0A6E3B3E035
:1002200001C01D92A937B107E1F70E9430010C947B
:100230003B220C9400001F920F920FB60F921124D4
:100240000F900FBE0F901F901895FC0120E030E03A
:1002500002C02F5F3F4F81918823D9F7C9010895CC
:10026000CCEFD0E1DEBFCDBFF8940E9464090E94BC
:10027000D20E8FEF84B985B92F980E94BE0981E80C
:1002800097E10E94090A85E69CE00E940E0A81E03F
:1002900090E00E94130ADE011196E2EEF2E083E0A4
:1002A00001900D928150E1F7CE0101960E94080E57
:1002B00080E091E00E94A40E81E191E00E949C0EFA
:1002C00082E491E00E94940E0E94DE0D4C0164E6EF
:1002D00070E00E94210A60E070E0C4010E944A0DB3
:1002E0003C0140E050E0BC01C4010E94420A22E10E
:1002F000A22E22E0B22ECC24DD2490E4E92EF12CB3
:1003000002E021E030E041E050E0B301C4010E948E
:10031000DF0C84E3A82E83E0B82E21E030E041E03A
:1003200050E0B301C4010E94170D10929403109283
:10033000930310929603109295030E94041B8FE77B
:1003400087B98AE288B90E940F0485E588B90E94BE
:100350000F0418B80E94580F0E9464090E94D70E1B
:100360007894FFCF0F931F93CF93DF93EC018134E9
:10037000910510F180919F039091A003892BE1F4E6
:10038000DF93CF938BE491E09F938F930E94FD1AAC
:1003900010929C0310929B03D0939E03C0939D03E5
:1003A00081E090E09093A00380939F03C0E4D0E0AD
:1003B0000F900F900F900F9068E08BE20E94A909B8
:1003C00000E010E00EC0E0919B03F0919C03E00F71
:1003D000F11FEB51FB4F608189E20E94A9090F5F79
:1003E0001F4F0C171D0779F7809193039091940389
:1003F000019749F467E08BE20E94A90910929403E7
:10040000109293030AC063E08BE20E94A90981E085
:1004100090E09093940380939303DF91CF911F9189
:100420000F910895CF93DF9380919F039091A00344
:10043000019709F04CC088E791E09F938F930E9449
:10044000FD1A20919B0330919C0380919D03909114
:100450009E030F900F9028173907C8F586E991E0A1
:100460009F938F930E94FD1AC0919D03D0919E038C
:1004700080919B0390919C03C81BD90B80919B0397
:1004800090919C03805C9F4F90939C0380939B036F
:100490000F900F90C134D1055CF08FEB91E09F93EA
:1004A0008F930E94FD1A80E490E00E94B2010DC07B
:1004B0008BED91E09F938F930E94FD1ACE010E94D5
:1004C000B2011092A00310929F030F900F90DF9142
:1004D000CF9108950F931F93CF93DF938C011092C8
:1004E0009C0310929B031092A00310929F032F9ADB
:1004F000FC018081282F22952F70C22FDD2799279C
:100500009F938F93DF93CF9388EE91E09F938F9388
:100510000E94FD1A8DB79EB706960FB6F8949EBF3F
:100520000FBE8DBFC430D10509F451C0C530D1050F
:1005300084F4C130D10569F1C230D1051CF4CD2B52
:10054000C1F077C0C230D10571F1239709F071C0B5
:1005500034C0C630D10509F44EC0C630D1050CF404
:1005600040C0C730D10509F450C0289709F061C0D8
:1005700056C0F8018081863041F48281813009F0D3
:100580006DC0C8010E948C1969C0C8010E94510F3A
:1005900065C088E092E09F938F930E94FD1AC80186
:1005A0000E94AA1359C08BE192E09F938F930E94FF
:1005B000FD1AC8010E940C154FC08FE292E09F9374
:1005C0008F930E94FD1AC8010E942C1645C083E437
:1005D00092E09F938F930E94FD1AC8010E94AA1770
:1005E0003BC087E592E09F938F930E94FD1AC8015C
:1005F0000E94CB1A31C08BE192E09F938F930E94AF
:10060000FD1AC8010E94F60527C08BE692E09F9371
:100610008F930E94FD1AC8010E94431F1DC08FE7DF
:1006200092E09F938F930E94FD1AC8010E94CA20F6
:1006300013C086E992E09F938F930E94FD1AF80100
:1006400080818093E50483E08093E6041092E704C0
:1006500083E090E00E94B2010F900F902F98DF91FD
:10066000CF911F910F9108950F931F93CF93DF9315
:10067000EC018C010F5F1F4F898199279F938F9306
:1006800083EA92E09F938F930E94FD1A80919503D5
:10069000909196030F900F900F900F90019791F506
:1006A00087EC92E09F938F930E94FD1A20E030E048
:1006B0000F900F90E0919703F0919803E20FF31FD2
:1006C000DE01A20FB31F8C91EB55FC4F80832F5F8F
:1006D0003F4F2034310571F7809197039091980333
:1006E000805C9F4F9093980380939703209197038A
:1006F000309198038091990390919A0328173907B4
:10070000F0F128C081ED92E09F938F930E94FD1A33
:10071000109298031092970320E030E00F900F9012
:10072000E0919703F0919803E20FF31FDE01A20F0F
:10073000B31F8C91EB55FC4F80832F5F3F4F2034CC
:10074000310571F73093980320939703F8012081C6
:10075000203448F4109296031092950385EA93E0B2
:100760000E946A020CC081E090E09093960380930F
:100770009503822F992790939A0380939903DF9191
:10078000CF911F910F9108951F920F920FB60F9264
:1007900011242F933F934F935F936F937F938F9386
:1007A0009F93AF93BF93EF93FF930E94230F80918A
:1007B0003F0386BDFF91EF91BF91AF919F918F91C4
:1007C0007F916F915F914F913F912F910F900FBE4D
:1007D0000F901F9018951F920F920FB60F92112431
:1007E0002F933F934F935F936F937F938F939F9339
:1007F000AF93BF93EF93FF930E94AC0EFF91EF91E5
:10080000BF91AF919F918F917F916F915F914F9128
:100810003F912F910F900FBE0F901F90189520E0E1
:1008200080E49CE90197F1F72F5F2931C9F708951A
:10083000882329F0813071F084E090E008958EE003
:100840008093690380936A0388E18093C10081E00B
:1008500090E008958EE080934E0380934F0388E1EB
:100860008093C90081E090E00895882329F08130C9
:1008700091F084E090E008951092690310926A0369
:100880001092C5001092C4001092C1001092C200D4
:1008900081E090E0089510924E0310924F03109261
:1008A000CD001092CC001092C9001092CA0081E0D5
:1008B00090E008950F93882329F0813041F084E07F
:1008C00090E00BC02093C5006093C40004C0209347
:1008D000CD006093CC0081E090E00F9108956230EC
:1008E00011F492E001C090E0882329F0813071F08A
:1008F00084E090E008958091C200990F990F990FBC
:10090000982B9093C20081E090E008958091CA00F6
:10091000990F990F990F982B9093CA0081E090E05E
:100920000895663061F0673019F0653019F404C03D
:1009300021E003C021E004C020E090E002C020E0FC
:1009400091E0882329F0813079F084E090E00895E7
:100950008091C200220F220F990F922B982B909317
:10096000C20081E090E008958091CA00220F220F1A
:10097000990F922B982B9093CA0081E090E00895F4
:10098000653439F06F3419F421E091E004C020E0BF
:1009900001C021E090E0882329F0813089F084E0D3
:1009A00090E008958091C2002295220F207E9295BA
:1009B000907F922B982B9093C20081E090E0089555
:1009C0008091CA002295220F207E9295907F922BD3
:1009D000982B9093CA0081E090E00895882329F035
:1009E000813061F084E090E008958091C00085FF3F
:1009F000FCCF6093C60081E090E008958091C8002C
:100A000085FFFCCF6093CE0081E090E00895FF92D7
:100A10000F931F93CF93DF93F82EEB018A0181E0B0
:100A20008F1548F484E090E00DC0F80161918F01CA
:100A30008F2D0E94EE042197FFEFCF3FDF07A9F72C
:100A400081E090E0DF91CF911F910F91FF90089589
:100A5000882329F0813051F084E090E0089580915E
:100A6000C00087FFFCCF8091C60006C08091C800FF
:100A700087FFFCCF8091CE0099270895FF920F93B6
:100A80001F93CF93DF93F82E8B0181E08F1518F41D
:100A900084E090E00EC0EA0107C08F2D0E94280577
:100AA000F80181938F0121971C161D06B4F381E094
:100AB00090E0DF91CF911F910F91FF9008957727DC
:100AC0000E9407058093E6041092E70483E090E01B
:100AD0000E94B20108950E9491048093E60410924E
:100AE000E70483E090E00E94B20108950E9491041F
:100AF0008093E6041092E70483E090E00E94B20144
:100B000008950E946F048093E6041092E70483E046
:100B100090E00E94B20108950F930E945A048093BE
:100B2000E6041092E70483E090E00E94B2010F9186
:100B300008950E9435048093E6041092E70483E050
:100B400090E00E94B20108950E9418048093E60488
:100B50001092E70483E090E00E94B2010895CF92E2
:100B6000DF92EF92FF920F931F93CF93DF93CDB756
:100B7000DEB78B01CDB6DEB62DB73EB7261B370BE1
:100B80000FB6F8943EBF0FBE2DBFEDB6FEB608946B
:100B9000E11CF11CAB01B7010E943E058093E60405
:100BA00020E030E00AC0F701E20FF31F8081F90175
:100BB000E951FB4F80832F5F3F4F201731079CF394
:100BC000F801E951FB4F1082C80103960E94B2015F
:100BD0000FB6F894DEBE0FBECDBEDF91CF911F9150
:100BE0000F91FF90EF90DF90CF9008950F93FC014D
:100BF00080818093E504843611F1853648F482368D
:100C0000B1F08336E0F4803651F0813681F50BC0C7
:100C1000873639F18836E9F0853649F515C0828185
:100C20000E94A4052DC082810E94990529C00681D9
:100C300025814481638182810E948C0521C063816A
:100C400082810E9481051CC0638182810E946B05A4
:100C500017C0AF014C5F5F4F638182810E945F05C7
:100C60000FC06381772782810E94AF0509C083E0AE
:100C70008093E6041092E70483E090E00E94B201C2
:100C80000F91089587E280934D0685E280934C068C
:100C900090E290934E0610924F0628E030E0309399
:100CA00051062093500683E28093590681E2809397
:100CB000580690935A0610925B0630935D06209377
:100CC0005C06089508956091650681E20E94A90975
:100CD000089568E08BE20E94A90961E188E20E9420
:100CE000A90968E08FE20E94A90961E18CE20E94F3
:100CF000A90961E08FE20E94A90910929403109261
:100D0000930365E083E20E94A90908950F931F935E
:100D10008C0160E480E20E94A909F80162816058B8
:100D200084E00E94A909F8018281809364061F91E2
:100D30000F9108950F931F93CF93DF93EC012885B4
:100D4000398512161306DCF58E819F818217930771
:100D50001CF568E083E20E94A90900E010E00FC0E2
:100D60008A859B85E80FF91F608181E20E94A909AD
:100D70008E819F8101969F838E830F5F1F4FEE812F
:100D8000FF8188859985083011051CF4E817F9075B
:100D90003CF3E817F90724F061E087E20E94A90913
:100DA0008B81813031F465E089810E94A9091B8221
:100DB00006C061E089810E94A90981E08B83DF91EF
:100DC000CF911F910F910895CF93DF93CDB7DEB7E9
:100DD00024970FB6F894DEBF0FBECDBFDC01FC0137
:100DE0002281338110925F0610925E0681E080932B
:100DF0005B06832F99278230D9F0833069F18130E7
:100E000009F057C080913806992790936106809326
:100E1000600688E396E0909363068093620686817D
:100E200097818034910509F044C088E090E029C0A2
:100E3000FD01868197819093610680936006E22F81
:100E4000FF27EE0FFF1F80914A0690914B06E80F97
:100E5000F91F8081918129C02223C1F0E22FFF2751
:100E6000EE0FFF1F8091A3039091A403E80FF91FD9
:100E70000190F081E02DF0936306E093620680819B
:100E80009927909361068093600613C094E099833C
:100E900083E08A8389E08B839C8384E090E0909355
:100EA000610680936006CE0101969093630680935D
:100EB000620688E596E00E949A0624960FB6F8949A
:100EC000DEBF0FBECDBFDF91CF910895CF93DF93EB
:100ED00082E20E948409C82FDD27C5FF1AC068E09E
:100EE00083E20E94A909C6FF10C020915E063091DE
:100EF0005F068091600690916106281739072CF4EF
:100F000088E596E00E949A0604C061E087E20E94AC
:100F1000A909DF91CF9108951F93CF93DF9388E0C4
:100F20000E948409182FC82FDD27C6FF18C060E073
:100F300085E00E94A90960E884E00E94A90960E0B8
:100F400080E20E94A90968E083E20E94A90961E0A9
:100F500087E20E94A90962E085E00E94A909C4FF16
:100F600004C060EC89E00E94A90917FF04C060ED8D
:100F700089E00E94A909DF91CF911F9108958AE02D
:100F80000E948409992780FF03C00E946607089584
:100F900081FF0DC08AE20E9484098091250681307C
:100FA00061F4E0912806F09129060995089582E3FD
:100FB0000E9484098AE30E94840908958EE00E94B9
:100FC000840968E08FE20E94A90961E08FE20E9433
:100FD000A909209160063091610680915C0690918C
:100FE0005D06821793075CF468E083E20E94A9091A
:100FF00061E087E20E94A90981E080935B06089581
:10100000AF92BF92CF92DF92EF92FF920F931F9316
:10101000CF93DF93CDB7DEB728970FB6F894DEBF36
:101020000FBECDBF86E20E94840986FF7EC08E017E
:101030000F5F1F4F580169E0C62ED12CCC0EDD1E6C
:1010400080914C060E948409F80181938F017501FB
:10105000EC15FD05A9F768E087E20E94A90968E0A0
:1010600083E20E94A90980E20E9484098F77682F99
:1010700080E20E94A9098981992780769070803248
:10108000910509F440C080349105D1F1892BF1F527
:10109000F50181818630D9F0873048F48130F1F153
:1010A0008130C8F08330D1F1853081F521C089309D
:1010B00019F18A3018F4883049F505C08A3071F189
:1010C0008B3021F520C0C5010E94630627C0C501F1
:1010D0000E94E40623C068E083E20E94A90961E05F
:1010E00081E20E94A90960E081E20E94A9090BC087
:1010F000C5010E94860612C0C5010E9469060EC085
:10110000C5010E94620965E083E206C080E20E9498
:1011100084098058682F80E20E94A909F701808124
:101120008823D1F465E083E215C0209160063091F8
:10113000610680915C0690915D068217930764F4C6
:10114000109261061092600668E083E20E94A9098D
:1011500061E087E20E94A90928960FB6F894DEBFE5
:101160000FBECDBFDF91CF911F910F91FF90EF90F8
:10117000DF90CF90BF90AF900895CF92DF92EF9223
:10118000FF920F931F93CF93DF93CDB7DEB7C05479
:10119000D0400FB6F894DEBF0FBECDBF8CE00E94EA
:1011A0008409992780FF03C00E9400087BC081FF4B
:1011B0002AC08EE20E9484098DE20E9484098983FC
:1011C0008E010F5F1F4F6801FFE3EF2EF12CE00E41
:1011D000F11E0F5F1F4F0E947209F80180830E15E8
:1011E0001F05B9F780913603813031F4E09139035E
:1011F000F0913A03C601099568E08FE20E94A909BF
:1012000061E08FE22BC082FF2CC086E30E9484093C
:1012100085E30E94840989838E010F5F1F4F680157
:10122000EFE3EE2EF12CE00EF11E0F5F1F4F0E9438
:101230007209F80180830E151F05B9F780913703F5
:10124000813031F4E0913B03F0913C03C6010995F4
:1012500068E087E30E94A90961E087E30E94A90989
:1012600021C083FF1FC08EE30E9484098E010F5F9F
:101270001F4F680171E4E72EF12CEC0EFD1E8DE38B
:101280000E948409F80181938F01EE15FF05B9F7DB
:1012900080913803813031F4E0913903F0913A03C1
:1012A000C6010995C05CDF4F0FB6F894DEBF0FBED4
:1012B000CDBFDF91CF911F910F91FF90EF90DF9005
:1012C000CF9008950895089581E080936A0080E1A9
:1012D0008DBB83B3876083BB84B3836084BB3F9A39
:1012E000479A089588B1805888B984B322E082274C
:1012F00084BB0000000080B198B1905898B994B3B5
:10130000922794BB992708959FEF91B982B988B12C
:10131000805888B984B395E0892784BB88B1805808
:1013200088B984B3892784BB000011B80E94720970
:101330009927089582B988B1805888B984B391E01B
:10134000892784BB88B1805888B984B3892784BB36
:10135000089582B98FEF81B988B1805888B984B374
:1013600095E0892784BB88B1805888B984B38927E0
:1013700084BB862F0E949A090895089582E1809384
:10138000380681E08093390680E191E090933B0636
:1013900080933A0610923C0610923D0610923E064B
:1013A00088E080933F06109241061092400610920A
:1013B000430610924206109245061092440610927F
:1013C000460610924706109248061092490610925F
:1013D00036031092370310923803109225061092AC
:1013E00026061092270610922F0610922E061092B3
:1013F000A2031092A10308959093410680934006A2
:10140000709343066093420650934506409344060A
:101410000895909341068093400608959093430663
:10142000809342060895909345068093440608955C
:1014300080933C06089580933D06089580933E0670
:101440000895CF93DF939C01CB01E0912E06F0919C
:101450002F0662E070E00E9414220FC0A081B181CB
:101460008281823039F4ED018D81992782179307AB
:1014700009F468870780F085E02D309779F7DF91D0
:10148000CF910895CF93DF939C01E0912E06F091C8
:101490002F0614C0A081B1818281843061F48481DF
:1014A00099278217930739F486819927861797071A
:1014B00011F4ED014B830780F085E02D309751F753
:1014C000DF91CF910895BF92CF92DF92EF92FF927A
:1014D0000F931F93CF93DF936C01162FF42EB22E30
:1014E000C0912E06D0912F062097A1F489E090E0BC
:1014F0000E941621FC0190932F0680932E06D18224
:10150000C082138310861782F282B4820583E6823A
:1015100015C0EC018F8198850097D9F789E090E09C
:101520000E941621FC0198878F83D182C082138389
:10153000F282B4820583E68210861782DF91CF9112
:101540001F910F91FF90EF90DF90CF90BF90089583
:10155000EF92FF921F93CF93DF937C01C091A10381
:10156000D091A203209711F011E012C085E090E025
:101570000E941621FC019093A2038093A103F182A3
:10158000E08212821482138210E012C01F5FEC010D
:101590008B819C810097D1F785E090E00E94162115
:1015A000FC019C838B83F182E0821283148213827C
:1015B000812F9927DF91CF911F91FF90EF90089590
:1015C000EF92FF920F931F93CF93DF93E091A103CC
:1015D000F091A20380E090E00380F481E02D019679
:1015E0003097D1F7880F991F0E9416219093A4037A
:1015F0008093A3030091A1031091A203E801E88066
:10160000F9808A81C82FDD27CC0FDD1F8091A303CD
:101610009091A403C80FD91FF701808199270E94D8
:1016200016219983888320E030E017C0E801EA8121
:10163000FF27EE0FFF1F8091A3039091A403E80FF3
:10164000F91F0190F081E02DE20FF31FD701A20FE7
:10165000B31F8C9180832F5F3F4FF70180819927C3
:10166000281739071CF3E8018B819C81009711F042
:101670008C01C4CFDF91CF911F910F91FF90EF901C
:1016800008954F925F926F927F928F929F92AF9246
:10169000BF92CF92DF92EF92FF920F931F93CF935F
:1016A000DF93E0912E06F0912F066624772409C07F
:1016B0008281823019F40894611C711C0780F085C6
:1016C000E02D3097A9F74301880C991CC4010E94B2
:1016D000162190934B0680934A06E1E0EE2EF12C02
:1016E000AA24BB2455C0E0912E06F0912F0679E084
:1016F000C72ED12C15C0A081B181848199278E1568
:101700009F0519F48381C80ED11CED018D818E15C2
:1017100021F48281823009F45D010780F085E02D9B
:10172000309749F700914A0610914B06025010403D
:10173000080D191DC6010E941621F80191838083AE
:1017400020E030E0E0914A06F0914B06E80DF91DEB
:1017500032970190F081E02DE20FF31FD501A20F27
:10176000B31F8C9180832F5F3F4F2930310551F794
:10177000E0914A06F0914B06E80DF91D3297019071
:10178000F081E02D8C2D875F82830894E11CF11C91
:101790006E147F040CF0A7CF61E0C62ED12C59E067
:1017A000A52EB12C4424552442E0842E912CA1C0B6
:1017B000A0912E06B0912F0612C0ED91FC911197C9
:1017C0008181823049F4858199278C159D0521F40A
:1017D0008481482E552405C0ED01AF81B88510974E
:1017E00061F731E0E32EF12C79C060912E06709103
:1017F0002F066DC0FB01C081D1818981843009F041
:1018000063C0868199278E159F0509F05DC084818C
:1018100099278C159D0509F057C0950140E050E0CF
:10182000E0914A06F0914B06E80DF91D32970190C0
:10183000F081E02DE20FF31FDE01A40FB51F8C91A4
:1018400080832F5F3F4F4F5F5F4F4930510541F716
:1018500089E090E0A80EB91EC0912E06D0912F0607
:1018600031C08A81853059F58C8199278C159D0569
:1018700031F58D8199278E159F0509F5088119810C
:10188000950140E050E0E0914A06F0914B06E80DEA
:10189000F91D32970190F081E02DE20FF31FD8017E
:1018A000A40FB51F8C9180832F5F3F4F4F5F5F4F19
:1018B0004730510541F7E7E0F0E0AE0EBF1E0F8064
:1018C000D885C02D209769F6EB016F817885611569
:1018D000710509F08FCF0894E11CF11C4E145F04D0
:1018E0000CF083CF0894C11CD11CE2E0F0E08E0E16
:1018F0009F1E6C147D040CF05BCFDF91CF911F9184
:101900000F91FF90EF90DF90CF90BF90AF909F909E
:101910008F907F906F905F904F9008956F927F921D
:101920008F929F92AF92BF92CF92DF92EF92FF92EF
:101930000F93CF93DF935C013B014901E0912E06A9
:10194000F0912F0616C0A081B18184819927A81635
:10195000B90661F4868199278615970539F4828145
:10196000843021F4ED018C818F5F8C830780F085BA
:10197000E02D309741F787E090E00E941621FC01AE
:1019800087E0808385E0818382820383F582E4821D
:10199000C682EE24062D2A2D45E067E0CF010E9485
:1019A000630ADF91CF910F91FF90EF90DF90CF907E
:1019B000BF90AF909F908F907F906F900895AF925F
:1019C000BF92CF92DF92EF92FF920F93FC01A1148E
:1019D000B10401F14230510571F04330510599F0E5
:1019E00041305105B9F481E080932506B092290673
:1019F000A09228060FC081E080932606B0922B06A5
:101A0000A0922A0607C081E080932706B0922D0697
:101A1000A0922C0620583F4FCF010E948E0C0F91B0
:101A2000FF90EF90DF90CF90BF90AF900895AF926E
:101A3000BF92CF92DF92EF92FF920F93FC01423060
:101A4000510571F04330510599F041305105B9F419
:101A500081E080933603B0923A03A09239030FC01D
:101A600081E080933703B0923C03A0923B0307C010
:101A700081E080933803B0923E03A0923D03CF01F2
:101A80000E948E0C0F91FF90EF90DF90CF90BF904F
:101A9000AF900895CF92DF92EF920F931F93CF9361
:101AA000DF936C018B01A0912E06B0912F06C0E050
:101AB000D0E014C02D913C911197F90185818C15CE
:101AC00051F4FD018281823031F4F90184818F5F0C
:101AD0008483C82FDD27FD01A781B085109751F7BA
:101AE00089E090E00E941621FC0189E0808384E077
:101AF00081830283138214821582168217821086D4
:101B0000EC2E00E02C2D44E069E0CF010E94630A36
:101B1000CE01DF91CF911F910F91EF90DF90CF9089
:101B20000895BF92CF92DF92EF92FF920F931F938F
:101B3000CF93DF936C017B01142FB22EA0912E0660
:101B4000B0912F06C0E0D0E014C02D913C911197C8
:101B5000F90185818C1551F4FD018281823031F4C7
:101B6000F90184818F5F8483C82FDD27FD01A78160
:101B7000B085109751F789E090E00E941621FC0192
:101B800089E0808384E08183E2821382148215835A
:101B9000B68207831086EC2E00E02C2D44E069E02D
:101BA000CF010E94630ACE01DF91CF911F910F9167
:101BB000FF90EF90DF90CF90BF900895EF920F933A
:101BC0001F93109149061F5F1093490689E090E02A
:101BD0000E941621FC0189E0808389E090E09383D4
:101BE000828382E0818314821583168280EA878350
:101BF0008AE18087EE2400E020E042E069E0CF0146
:101C00000E94630A812F99271F910F91EF900895E9
:101C1000CF93DF93EC01FC0101900020E9F7E81B72
:101C2000F90BCF01880F991F0E9416219C01FE011C
:101C300001900020E9F7EC1BFD0BEE0FFF1FDC010C
:101C4000EC9383E0F901818340E050E009C0FE019C
:101C5000E40FF51F80818C93FD0111824F5F5F4F70
:101C60001296FE0101900020E9F73197EC1BFD0B65
:101C70004E175F0760F3C9010E94A80A9927DF91F8
:101C8000CF910895EF92FF920F931F93CF93DF931D
:101C90008C017B01CA010E94080E9C01E0912E0676
:101CA000F0912F0614C0A081B1818281843061F44B
:101CB000848199278017910739F4868199278E1599
:101CC0009F0511F4ED0128870780F085E02D3097FE
:101CD00051F7DF91CF911F910F91FF90EF900895F1
:101CE0000F931F93CF93DF938C01CB010E94080EBB
:101CF0009C01E0912E06F0912F060FC0A081B181CA
:101D00008281823039F4ED018D8199278017910706
:101D100009F42E830780F085E02D309779F7DF9165
:101D2000CF911F910F9108950E94080E1816190661
:101D300014F48093480608950E94080E1816190698
:101D400014F48093470608950E94080E1816190689
:101D500014F48093460608951F9386E00E94840938
:101D6000992786FF03C00E94BD080EC082FF03C0F2
:101D70000E94BF0709C081FF03C00E948C0704C0F6
:101D800084FF02C00E94DE0787E00E948409182FAA
:101D900060E087E00E94A909612F87E00E94A909FD
:101DA0001F91089562E081E00E94A90908950E94B0
:101DB000410B0E94E00A0E94420661E080E00E941E
:101DC000A90980E00E94840980FDFBCF62E081E0E8
:101DD0000E94A90960E884E00E94A90960E480E209
:101DE0000E94A90968E083E20E94A90969E087E2EC
:101DF0000E94A9096FE08DE00E94A9096FE08BE0C5
:101E00000E94A90968ED89E00E94A90963E38FE0B7
:101E10000E94A90966ED87E00E94A90962E085E0B9
:101E20000E94A9096CEC80E00E94A90908958EEC3B
:101E300080933F0381E080936E0080913F0386BDD5
:101E400083E084BD08950895089583E08093E504B8
:101E500081E08093E6048BE08093E7042FE62093F3
:101E6000E80493E69093E90484E78093EA042093DE
:101E7000EB049093EC0481E68093ED048EE680936E
:101E8000EE048FE58093EF0480E38093F00481E318
:101E90008093F1041092F2048EE090E00E94B2016F
:101EA0000895FC018081833011F40E94250F08956C
:101EB0001F9311E0812F0E94631060E0812F0E9428
:101EC00037111F5F1431B1F718E1812F0E946310A1
:101ED00060E0812F0E9437111F5F1B32B1F71F9105
:101EE0000895CF93DF93DC01EC01EA81FB8121911E
:101EF0008E81815019F48981E81BF109ED01FB8382
:101F0000EA838E839FB7F8948C9181508C939FBF06
:101F1000822F9927DF91CF910895FC01108275835C
:101F20006483738362834183478346830895CF9399
:101F3000DF93DC019C91ED018981981718F080E016
:101F400090E016C0ED01EC81FD8161938F8181509D
:101F500019F48981E81BF109ED018F83FD83EC837E
:101F60009FB7F8948C918F5F8C939FBF81E090E036
:101F7000DF91CF910895FC0180818823E9F3CF019F
:101F80000E94710F99270895FC018081882319F41C
:101F90008FEF9FEF0895CF010E94710F9927089549
:101FA00081E090E0089581E090E0089581E090E084
:101FB000089581E090E00895CF93DF93CDB7DEB729
:101FC00022970FB6F894DEBF0FBECDBF982F815079
:101FD000833120F08751833108F066C0E92FFF2755
:101FE000E15CFC4F82E08183892F9927AA27BB27D8
:101FF000FC013197EC32F10508F056C0E65BFF4F6B
:10200000EE0FFF1F0590F491E02D09946D9A43C0E7
:102010006E9A45C06F9A3FC0209A41C0219A3BC03A
:10202000229A3DC0239A37C0249A39C0259A33C0DA
:10203000269A35C0279A2FC0509A31C0519A2BC08A
:10204000529A2DC0539A27C0549A29C0559A23C03A
:10205000569A25C0579A1FC0389A21C0399A1BC07A
:102060003A9A1DC03B9A17C03C9A19C0879A13C070
:10207000869A15C0859A0FC0849A11C0839A0BC0A6
:10208000829A0DC0699A07C0689A09C0689A03C00D
:10209000699A05C06A9A81E090E008C06B9AE1E015
:1020A000F0E0FA83E98304C084E090E09A838983B6
:1020B00089819A8122960FB6F894DEBF0FBECDBFFC
:1020C000DF91CF910895982F8150833130F087515F
:1020D000833118F084E090E00895892F0E94DC0F8E
:1020E00081E090E00895CF93DF93CDB7DEB72297DC
:1020F0000FB6F894DEBF0FBECDBF982F815083314D
:1021000020F08751833108F066C0E92FFF27E15C9A
:10211000FC4F81E08183892F9927AA27BB27FC01E7
:102120003197EC32F10508F056C0EA58FF4FEE0F38
:10213000FF1F0590F491E02D09946D9843C06E98AF
:1021400045C06F983FC0209841C021983BC022985D
:102150003DC0239837C0249839C0259833C02698AD
:1021600035C027982FC0509831C051982BC0529835
:102170002DC0539827C0549829C0559823C056980D
:1021800025C057981FC0389821C039981BC03A986D
:102190001DC03B9817C03C9819C0879813C08698FB
:1021A00015C085980FC0849811C083980BC0829881
:1021B0000DC0699807C0689809C0689803C06998FD
:1021C00005C06A9881E090E008C06B98E1E0F0E01B
:1021D000FA83E98304C084E090E09A83898389814B
:1021E0009A8122960FB6F894DEBF0FBECDBFDF9165
:1021F000CF910895FB011082833091F0843028F450
:10220000813051F0823029F409C0843059F0853092
:1022100059F085E090E0089583B107C086B105C00C
:1022200089B103C08CB101C08FB1808381E090E09F
:102230000895833091F0843028F4813051F0823059
:1022400029F409C0843059F0853069F084E090E0C9
:10225000089565B905C068B903C06BB901C06EB90E
:1022600081E090E0089561BB81E090E00895982FAF
:10227000E82FFF27E15CFC4F8181823019F086E076
:1022800090E00895892F9927AA27BB27FC01319751
:10229000EC32F10540F4EE55FF4FEE0FFF1F0590B5
:1022A000F491E02D099484E090E00895662311F004
:1022B000759AC5C07598C3C0662311F0769ABFC0E1
:1022C0007698BDC0662311F0779AB9C07798B7C0E9
:1022D000662311F0289AB3C02898B1C0662311F084
:1022E000299AADC02998ABC0662311F02A9AA7C0DD
:1022F0002A98A5C0662311F02B9AA1C02B989FC0E5
:10230000662311F02C9A9BC02C9899C0662311F07B
:102310002D9A95C02D9893C0662311F02E9A8FC0E8
:102320002E988DC0662311F02F9A89C02F9887C0F0
:10233000662311F0589A83C0589881C0662311F023
:10234000599A7DC059987BC0662311F05A9A77C07C
:102350005A9875C0662311F05B9A71C05B986FC084
:10236000662311F05C9A6BC05C9869C0662311F01B
:102370005D9A65C05D9863C0662311F05E9A5FC088
:102380005E985DC0662311F05F9A59C05F9857C090
:10239000662311F0409A53C0409851C0662311F053
:1023A000419A4DC041984BC0662311F0429A47C0F4
:1023B000429845C0662311F0439A41C043983FC0FC
:1023C000662311F0449A3BC0449839C0662311F04B
:1023D0008F9A35C08F9833C0662311F08E9A2FC024
:1023E0008E982DC0662311F08D9A29C08D9827C034
:1023F000662311F08C9A23C08C9821C0662311F0BB
:102400008B9A1DC08B981BC0662311F08A9A17C047
:102410008A9815C0662311F0709A11C070980FC089
:10242000662311F0719A0BC0719809C0662311F0F0
:10243000729A05C0729803C0662321F0739A81E0F6
:1024400090E00895739881E090E008951F93182F0D
:102450008150833130F08751833118F084E090E06F
:102460000FC0E12FFF27E15CFC4F83E08183812FC8
:102470000E94DC0F61E0812F0E94371181E090E023
:102480001F910895CF93DF93982FEB011882E82FC7
:10249000FF27E15CFC4F8181813019F086E090E0FC
:1024A0007DC0892F9927AA27BB27FC013197EC32E1
:1024B000F10540F4E253FF4FEE0FFF1F0590F4913A
:1024C000E02D099484E090E069C0659B65C062C01E
:1024D000669B62C05FC0679B5FC05CC0189B5CC0AE
:1024E00059C0199B59C056C01A9B56C053C01B9B5C
:1024F00053C050C01C9B50C04DC01D9B4DC04AC016
:102500001E9B4AC047C01F9B47C044C0489B44C055
:1025100041C0499B41C03EC04A9B3EC03BC04B9B13
:102520003BC038C04C9B38C035C04D9B35C032C015
:102530004E9B32C02FC04F9B2FC02CC0309B2CC055
:1025400029C0319B29C026C0329B26C023C0339BA3
:1025500023C020C0349B20C01DC07F9B1DC01AC05B
:102560007E9B1AC017C07D9B17C014C07C9B14C0F3
:1025700011C07B9B11C00EC07A9B0EC00BC0609B2C
:102580000BC008C0619B08C005C0629B05C002C0AB
:10259000639B02C081E0888381E090E0DF91CF916E
:1025A0000895CF93DF93CDB7DEB721970FB6F89498
:1025B000DEBF0FBECDBF9BE19093E504BE016F5F10
:1025C0007F4F0E9442128093E60489818093E70442
:1025D0001092E80484E090E00E94B20121960FB6C8
:1025E000F894DEBF0FBECDBFDF91CF9108959AE181
:1025F0009093E5040E9437118093E6041092E7045B
:1026000083E090E00E94B201089598E19093E50480
:102610000E9419118093E6041092E70483E090E091
:102620000E94B2010895982F89E18093E5049330C8
:1026300099F0943028F4913059F0923029F40AC07E
:10264000943061F0953061F085E090E020E00BC0BF
:1026500023B107C026B105C029B103C02CB101C008
:102660002FB181E090E08093E6042093E70410927C
:10267000E80484E090E00E94B201089597E190930D
:10268000E5040E9426128093E6041092E70483E09A
:1026900090E00E94B201089595E19093E5040E94B4
:1026A00073108093E6041092E70483E090E00E94A8
:1026B000B201089596E19093E5040E94DC0F8093A7
:1026C000E6041092E70483E090E00E94B2010895CE
:1026D00084E18093E50481E08093E6041092E704AE
:1026E00083E090E00E94B201089582E18093E504C6
:1026F00081E08093E6041092E70483E090E00E947A
:10270000B201089583E18093E50481E08093E604BB
:102710001092E70483E090E00E94B201089580E106
:102720008093E50481E08093E6041092E70483E05F
:1027300090E00E94B201089591E19093E5040E9417
:1027400063108093E6041092E70483E090E00E9417
:10275000B2010895FC0180818531C9F1863180F490
:10276000823131F1833130F48031D1F0813109F09F
:102770004CC01AC0833109F1843109F046C022C02F
:10278000883189F1893128F4863129F18731E9F5D9
:1027900026C08A3189F18A3158F18B31B1F531C0C7
:1027A00082810E948F13089582810E949C13089554
:1027B000638182810E9475130895638182810E94E2
:1027C00082130895638182810E9468130895828133
:1027D0000E944C13089582810E945A1308958281A9
:1027E0000E943E130895638182810E94051308951B
:1027F00082810E9413130895638182810E94F712DF
:10280000089582810E94D11208958093E50483E0A7
:102810008093E6041092E70483E090E00E94B20106
:102820000895E82F8152883018F084E090E00895F0
:10283000FF27E15CFC4F84E0818381E090E0089514
:10284000E82FFF27E15CFC4F8181843019F084E0A0
:1028500090E00895118281E090E0089510927C004C
:10286000823039F0833069F0813041F082E090E0CD
:10287000089580917C00806480937C0081E090E0EA
:10288000089580917C00806C80937C0081E090E0D2
:10289000089593E890937A0090917C00907F982B14
:1028A00090937C0080917A00806480937A0080917C
:1028B0007A0086FDFCCF809178009091790020E02D
:1028C00030E040E050E080917A00806480937A00AC
:1028D00080917A0086FDFCCF8091780090917900FC
:1028E000480F591F2F5F3F4F2430310561F780910A
:1028F0007A008F7780937A00CA019695879596958E
:1029000087950895CF93DF93EB0119821882282FC2
:102910003327F901E15CFC4F8181843019F086E0B6
:1029200090E00AC088E290E0821B930B0E94491459
:102930009983888381E090E0DF91CF91089593E2BD
:102940009093E5040E942E148093E6041092E7040D
:1029500083E090E00E94B2010895CF93DF93CDB75A
:10296000DEB722970FB6F894DEBF0FBECDBF92E25E
:102970009093E504BE016F5F7F4F0E9482148093A5
:10298000E60429813A81832F99278093E7042093D5
:10299000E8041092E90485E090E00E94B2012296DA
:1029A0000FB6F894DEBF0FBECDBFDF91CF91089573
:1029B00091E29093E504E82FFF27E15CFC4F8181D1
:1029C000843019F084E090E003C0118281E090E04F
:1029D0008093E6041092E70483E090E00E94B20145
:1029E0000895E82F80E28093E5048E2F815288308D
:1029F00018F084E090E007C0FF27E15CFC4F84E022
:102A0000818381E090E08093E6041092E70483E004
:102A100090E00E94B2010895FC018081813271F042
:102A2000823218F48032B1F405C0823259F0833218
:102A300089F40CC082810E94F114089582810E9461
:102A4000D814089582810E94AD14089582810E9455
:102A50009F1408958093E50483E08093E604109228
:102A6000E70483E090E00E94B2010895ECEBF0E00F
:102A70008081846080838BE080934C038CE0809322
:102A80004D0381E090E00895ECEBF0E080818B7FD6
:102A9000808310924C0310924D0381E090E00895E2
:102AA0008093B800E9EBF0E080818C7F80838081A7
:102AB000808381E090E008958091B9009927887F14
:102AC000907008958091B90084EA8093BC00809151
:102AD000BC0087FFFCCF81E090E0089584E98093FB
:102AE000BC008091BC0084FDFCCF81E090E00895A3
:102AF000AC0120E030E00FC0FA01E20FF31F80814B
:102B00008093BB0084E88093BC008091BC0087FF69
:102B1000FCCF2F5F3F4F2617370774F3089584E8E3
:102B20008093BC008091BC0087FFFCCF8091BB00EC
:102B30009927089585E38093E50481E08093E60476
:102B400020E030E00FC084E88093BC008091BC009E
:102B500087FFFCCF8091BB00F901E951FB4F8083D7
:102B60002F5F3F4F2617370774F3FB01E951FB4FE7
:102B70001082CB0103960E94B20108959B01BC0113
:102B8000C9010E94781581E08093E6041092E70461
:102B900083E090E00E94B201089584E98093BC0034
:102BA0008091BC0084FDFCCF81E08093E60410920C
:102BB000E70483E090E00E94B20108958091B9009B
:102BC00084EA8093BC008091BC0087FFFCCF81E049
:102BD0008093E6041092E70483E090E00E94B20143
:102BE00008958093B800E9EBF0E080818C7F8083CA
:102BF0008081808381E08093E6041092E70483E083
:102C000090E00E94B2010895ECEBF0E080818B7FB0
:102C1000808310924C0310924D0381E08093E60470
:102C20001092E70483E090E00E94B2010895ECEB7B
:102C3000F0E08081846080838BE080934C038CE0A3
:102C400080934D0381E08093E6041092E70483E0D3
:102C500090E00E94B2010895FC0180818093E50418
:102C60008433D1F0853338F4813379F0823381F0C5
:102C7000803331F507C08633E9F08633A0F087331F
:102C8000F9F41BC00E94171608950E9404160895B7
:102C900082810E94F115089582813396BF019927A0
:102CA0000E94BE15089563817727828199270E942B
:102CB0009A1508950E94DE1508950E94CD15089575
:102CC00083E08093E6041092E70483E090E00E94A2
:102CD000B2010895782F613079F0613050F06230A0
:102CE00021F0633009F059C002C061E003C061E027
:102CF00004C060E030E002C060E031E04330D9F071
:102D0000443028F4413089F0423090F40CC0453012
:102D100031F04530A0F0463009F03FC002C040E03D
:102D200005C040E006C041E007C041E050E005C0FA
:102D300041E050E006C040E051E020E003C040E048
:102D400051E021E0239884B1866084B985B1817F08
:102D500085B980E090E0772311F081E090E075E0A4
:102D6000880F991F7A95E1F78065660F660F660FE9
:102D7000682B330F330F362B352B440F432B4CBDB1
:102D80002DBD88E0809345038AE08093460389E067
:102D90008093470381E090E0089582E090E00895F9
:102DA0001CBC1DBC109245031092460310924703B1
:102DB00081E090E00895AC0120E030E009C0E60F2A
:102DC000F71F80818EBD0DB407FEFDCF2F5F3F4FF3
:102DD000E22FFF27E417F50794F381E090E00895D0
:102DE000DC0120E030E040E050E015C01EBC09C02E
:102DF00083E0493E58071CF088E090E008954F5F5B
:102E00005F4F0DB407FEF4CFFB01E20FF31F8EB549
:102E100080832F5F3F4F2A173B0744F381E090E008
:102E20000895CF93DF93EC01A0E0B0E020E030E024
:102E300018C0FE01E20FF31F80818EBD08C01196FD
:102E400083E0A93EB8071CF088E090E00FC00DB405
:102E500007FEF5CFFB01E20FF31F8EB580832F5FD6
:102E60003F4F241735072CF381E090E0DF91CF919D
:102E70000895EF92FF920F931F938B01E5EEEE2ED4
:102E8000E4E0FE2E23E42093E504B7016E5F7F4F5C
:102E9000A8010E9411178093E6040E5F1F4FE00EF9
:102EA000F11EF7011082C80101960E94B2011F9124
:102EB0000F91FF90EF900895EF92FF920F931F9361
:102EC0008C01F5EEEF2EF4E0FF2E84E48093E50410
:102ED000B7016E5F7F4FC8010E94F0168093E60431
:102EE0000E5F1F4FE00EF11EF7011082C801019620
:102EF0000E94B2011F910F91FF90EF90089593E40B
:102F00009093E50499270E94DB168093E6041092C3
:102F1000E70483E090E00E94B201089581E4809389
:102F2000E5040E94D0168093E6041092E70483E043
:102F300090E00E94B201089590E49093E5040E940D
:102F40006A168093E6041092E70483E090E00E9402
:102F5000B2010895CF93DF93EC0188818334A9F007
:102F6000843428F4803441F0813409F50BC0843472
:102F700099F08534E1F414C04C816B818A810E9400
:102F80009C1720C00E948E171DC0BE016D5F7F4F31
:102F90008A810E947F1716C08A8199270E945C1738
:102FA0006A817727CE0103960E9439170BC0809360
:102FB000E50483E08093E6041092E70483E090E068
:102FC0000E94B201DF91CF910895209A219A229A0E
:102FD0002398249A259A2C982D9881E08093500369
:102FE00082E080935103809352038093530381E0E6
:102FF00090E00895109250031092510310925203E2
:103000001092530381E090E00895289829982A9817
:1030100080E29EE40197F1F7289A8AE0982F9A952A
:10302000F1F72A9A299A8A95F1F70895282F299875
:1030300087FD02C02A9801C02A9A8AE0982F9A95A3
:10304000F1F7299A8A95F1F7299826FF02C02A9A62
:1030500001C02A988AE0982F9A95F1F7299A8A95C3
:10306000F1F70895282F220F30E0299827FF02C09A
:103070002A9A01C02A988AE0982F9A95F1F7299AFE
:103080008A95F1F73F5F373011F0220FEECF0895A8
:10309000282F30E0299827FF02C02A9A01C02A98D9
:1030A0008AE0982F9A95F1F7299A8A95F1F73F5F70
:1030B000383011F0220FEECF089529982A988AE02F
:1030C000982F9A95F1F7299A982F9A95F1F72998C0
:1030D0002898982F9A95F1F7299A982F9A95F1F7B1
:1030E00029988A95F1F7289A80E090E00895299828
:1030F00028982A982B9A08950E94051880E30E9428
:10310000161880E60E94321808950E94051880E083
:103110000E94161880E00E9432180E9477180895C5
:103120000F931F93182F062F0E94051880E40E940A
:103130001618812F0E943218802F0E94481881E0B3
:1031400090E01F910F9108951F93182F0E9405186A
:1031500080EC0E941618812F0E9432180E945D1880
:1031600099271F91089529988AE08A95F1F72A985E
:1031700090E030E0990F299A2AE0822F8A95F1F7A2
:1031800029981B999F5F822F8A95F1F73F5F38300E
:1031900089F72898299A822F8A95F1F7289A2998F1
:1031A0002A95F1F7892F992708951F93182F0E94C8
:1031B000051880E80E941618812F0E9432180E947C
:1031C000B31899271F910895DF92EF92FF920F9302
:1031D0001F93CF93DF93D82E7B018A01C0E0D0E00C
:1031E00009C08D2D8C0F0E94D518F801EC0FFD1F22
:1031F00080832196CE15DF05A1F781E090E0DF9175
:10320000CF911F910F91FF90EF90DF9008950F9352
:103210001F93082F162F0E947C18612F802F0E9469
:10322000901881E090E01F910F910895DF92EF9246
:10323000FF920F931F93CF93DF93D82E7B018A01C8
:10324000C0E0D0E009C0F801EC0FFD1F60818D2DBA
:103250008C0F0E9407192196CE15DF05A1F781E09A
:1032600090E0DF91CF911F910F91FF90EF90DF9051
:10327000089594E09093E5040E9416198093E60463
:103280001092E70483E090E00E94B2010895EF926B
:10329000FF920F931F938B0195EEE92E94E0F92E88
:1032A00093E09093E504A7014E5F5F4F0E94E418FE
:1032B0008093E6040E5F1F4FE00EF11EF7011082AF
:1032C000C80101960E94B2011F910F91FF90EF90EB
:1032D000089582E08093E504109250031092510308
:1032E000109252031092530381E08093E6041092EF
:1032F000E70483E090E00E94B201089581E08093AA
:10330000E5040E94E5178093E6041092E70483E049
:1033100090E00E94B2010895FC018381823069F03F
:10332000833018F48130F1F405C0833049F08430E3
:10333000C9F40FC00E947E1908950E94691908956A
:10334000AF014A5F5F4F6581772784810E944719EB
:103350000895AF014A5F5F4F6581772784810E949E
:103360003919089580818093E50483E08093E60411
:103370001092E70483E090E00E94B20108951F924A
:103380000F920FB60F9211240F900FBE0F901F9047
:1033900018959C010897029718F084E090E0089532
:1033A000F901E15CFC4F8DE0818328303105B1F0FB
:1033B0002930310519F087E090E00895259A81E0E1
:1033C00090E0909389008093880081E8809380004A
:1033D00089E08093810081E090E00895249A81E063
:1033E0008093B30089E68093B00081E090E0089577
:1033F0009C01FC01E15CFC4F81818D3019F086E07D
:1034000090E008952830310539F12930310519F05F
:1034100087E090E0089563307105B1F06430710584
:1034200044F46130710561F06230710509F040C00B
:1034300009C06430710551F065307105C9F508C0E7
:1034400081E007C082E005C083E003C084E001C0E2
:1034500085E08093810029C064307105E9F0653012
:10346000710554F46230710599F06330710594F47C
:1034700061307105E9F40AC06630710589F0663083
:10348000710564F06730710599F40CC089E60BC0D2
:103490008AE609C08BE607C08CE605C08DE603C04E
:1034A0008EE601C08FE68093B00081E090E0089541
:1034B00081E090E008959C01FC01E15CFC4F81817A
:1034C0008D3019F086E090E008952830310569F0DC
:1034D0002930310519F087E090E008957093890054
:1034E0006093880081E090E008956093B30081E0EC
:1034F00090E0089523E52093E5040E945B1A8093F1
:10350000E6041092E70483E090E00E94B20108957F
:1035100022E52093E5040E94F8198093E6041092B6
:10352000E70483E090E00E94B201089520E5209333
:10353000E5040E94C9198093E6041092E70483E031
:1035400090E00E94B2010895FC01E15CFC4F118201
:103550008830910531F08930910531F086E090E0B6
:1035600008951092B00004C0109281001092800063
:103570000E94DC0F81E090E0089521E52093E504AE
:103580000E94A41A8093E6041092E70483E090E07E
:103590000E94B2010895FC018081813579F0823565
:1035A00018F48035F1F405C0823569F08335C9F42B
:1035B00011C0828199270E94961A089582819927C5
:1035C0000E94BD1A089563817727828199270E94FE
:1035D000881A089563817727828199270E947A1A31
:1035E00008958093E50483E08093E6041092E70455
:1035F00083E090E00E94B2010895CF93DF93CDB7AE
:10360000DEB7DF91CF910895089581E090E00895AD
:1036100008958A3310F4805301C087556A3310F43B
:10362000605301C067556F708295807F682B862F2D
:103630009927089508958230A1F0833028F48823D3
:1036400061F0813039F40BC0843079F0843058F067
:103650008530B9F080E090E0089582E107C08EE007
:1036600005C088E003C086E001C082E08093E200EC
:103670008CE08093E30087E38093E40081E090E0B6
:1036800008951092E2008CE08093E30087E380933A
:10369000E40081E090E00895813091F0813038F0CD
:1036A0008230E1F0833061F180E090E00895809114
:1036B000DB008F778093DB008091DB008F7D16C06D
:1036C0008091DB0080688093DB008091DB008F7D40
:1036D0008093DB008091DB0080610DC08091DB0076
:1036E00080688093DB008091DB0080628093DB0048
:1036F0008091DB008F7E8093DB0081E090E0089575
:103700008091DB0080688093DB008091DB00806229
:103710008093DB008091DB0080618093DB0081E09F
:1037200090E008951F93982F162F8FE080935103F8
:103730008093520310927406442319F081E0809321
:103740007406109268061092690610926A0610922A
:103750006B06ECE6F6E0119286E0E437F807D9F75D
:1037600020E030E0822F8295807F8093ED001092E0
:10377000EE001092EF002F5F3F4F2F30310591F791
:10378000892F0E941B1B892B89F0812F0E944C1BC3
:10379000892B61F08091D80082608093D80080915D
:1037A000D90082FFFCCF81E090E002C082E090E08F
:1037B0001F9108958295807F8093ED0008959B016D
:1037C000AC0180917406882381F4822F8295880F42
:1037D000807E8093F60063E0569547953795279550
:1037E0006A95D1F72093F7000895DA01C90153E0F3
:1037F000880F991FAA1FBB1F5A95D1F78760809326
:10380000F400292F3A2F4B2F55272093F5009D01C7
:10381000442755272093F6008B2F9927AA27BB27EB
:103820008093F7000895EF92FF920F931F9380917A
:1038300074068823C1F42091F20022952695277002
:103840003327442755278091F300992703E0880FF9
:10385000991F0A95E1F77C0100271127E22AF32A34
:10386000042B152B33C02091F3008091F200E090DF
:10387000F1006091F0009927AA27BB27DC01992766
:103880008827332744275527522F442733272227B9
:10389000822B932BA42BB52BFF2400271127102F4D
:1038A0000F2DFE2CEE248E299F29A02BB12BE62E66
:1038B000FF2400271127E82AF92A0A2B1B2B73E083
:1038C00016950795F794E7947A95D1F7C801B70153
:1038D0001F910F91FF90EF9008959B01AC01809193
:1038E0007406882371F4822F8295880F807E8093DE
:1038F000F200E3E05695479537952795EA95D1F77D
:1039000025C073E0220F331F441F551F7A95D1F74E
:103910008091F0009927AA27BB2787709070A0702C
:10392000B070282B392B4A2B5B2B2093F000BB2740
:10393000A52F942F832F8093F100CA01AA27BB27BC
:103940008093F200252F3327442755272093F30037
:103950000895982F80917406882321F08091EF00BC
:10396000806103C08091EF008F7E8093EF009230E2
:1039700091F1933028F4992359F0913031F422C019
:103980009330E1F1943009F450C080E090E0089564
:103990008091EF008F7B8093EF008091EF008F7715
:1039A0008093EF008091EF008F7D8093EF008091F6
:1039B000F0008B7F8093F0008091F4008B7F8093E8
:1039C000F40030C08091EF0080648093EF0080911C
:1039D000EF008F771BC08091EF008F778093EF000F
:1039E0008091EF0080648093EF008091EF008F7DE5
:1039F0008093EF008091F000846012C08091EF000E
:103A00008F7B8093EF008091EF0080688093EF00C0
:103A10008091EF008F7D8093EF008091F0008B7F8D
:103A20008093F00081E090E008958091EF008F7B1B
:103A30008093EF008091EF0080688093EF00809189
:103A4000EF0080628093EF008091F00084608093AB
:103A5000F00081E090E008959F92AF92BF92CF92E4
:103A6000DF92EF92FF920F931F93E82F962E59014A
:103A70006A01C801B7012E2F2295207F2093ED0007
:103A80004091DE00FF27EB51FD4F21E030E0008048
:103A900002C0220F331F0A94E2F7422B4093DE004C
:103AA0000E94DF1BC601B5010E946D1C892D0E947A
:103AB000A91C892B19F482E090E002C081E090E01B
:103AC0001F910F91FF90EF90DF90CF90BF90AF903C
:103AD0009F9008958091EF0087FD04C08091EF00D2
:103AE00086FF3CC08091EF0087FD0AC08091EF0007
:103AF00086FF06C08091F00082FD02C081E02FC0E9
:103B00008091EF0087FD0AC08091EF0086FF06C01C
:103B10008091F00082FF02C082E021C08091EF001E
:103B200087FF0AC08091EF0086FD06C08091F000FB
:103B300082FD02C083E013C08091EF0087FF0EC0BA
:103B40008091EF0086FD0AC08091EF0085FF06C0DE
:103B50008091F00082FF02C084E001C080E09927DC
:103B60000895982F893008F098E08091EF00807FC9
:103B7000892B8093EF00FB0120E004C081918093AA
:103B8000FA002F5F2917D1F70895EF92FF920F9354
:103B90001F93F62E8A018295807F8093ED000E940C
:103BA0006A1DE82EB8018F2D0E94B11D81E00E9490
:103BB000A91C8091EE0086FFFCCF8091EE008F7BE8
:103BC0008093EE008E2D0E94A91C81E090E01F9151
:103BD0000F91FF90EF900895FF920F931F93F62E91
:103BE0008A018295807F8093ED0084E00E94A91C69
:103BF000B8018F2D0E94B11D1F910F91FF90089564
:103C0000AC0120E030E0FA01E20FF31F8091FA00EE
:103C100080832F5F3F4F28303105A9F70895AEED1F
:103C2000B0E02C91E5EEF2E0E80FF11D81E090E0CC
:103C3000008002C0880F991F0A94E2F7282B2C936A
:103C40000895AEEDB0E02C91E5EEF2E0E80FF11D45
:103C500081E090E0008002C0880F991F0A94E2F78B
:103C6000809582238C9308952091E0008091E1005B
:103C70009927982F88273327822B932B009779F049
:103C800020E030E002C096958795422F2F5F3F4F8E
:103C900080FFF9CF4F3018F4842F992708958FEFC4
:103CA00090E00895982F9295907F9093ED000E9458
:103CB000211E80E00E94A91C81E090E00895CF932E
:103CC000DF931092510310925203C0E0D0E08C2F8A
:103CD0000E94521E2196CF30D105C9F78091D8009D
:103CE0008D7F8093D8008091D90082FDFCCF81E048
:103CF00090E0DF91CF9108951F938295807F80930C
:103D0000ED000E946A1D182F82E00E94A91C80917C
:103D1000EE0086FFFCCF8091EE008F7B8093EE005B
:103D2000812F0E94A91C81E090E01F91089586E7F1
:103D30008093E50481E08093E60480916806909189
:103D40006906A0916A06B0916B068093E704292F5B
:103D50003A2F4B2F55272093E8049D0144275527E0
:103D60002093E9048B2F9927AA27BB278093EA0485
:103D7000109268061092690610926A0610926B06FD
:103D8000ACE6B6E026E030E08C91F901EB51FB4F58
:103D900080831D922F5F3F4F2E303105A9F710927F
:103DA000F3048FE090E00E94B201089595E79093AC
:103DB000E5040E947C1E8093E6041092E70483E0F1
:103DC00090E00E94B201089594E79093E5040E9468
:103DD000521E8093E6041092E70483E090E00E9474
:103DE000B201089592E79093E5040E94C51D809367
:103DF000E6041092E70483E090E00E94B201089587
:103E0000EF92FF920F931F9393E79093E5040E9424
:103E10002C1D8093E6041092E70483E090E00E945A
:103E2000B2011F910F91FF90EF9008950E94EC1D39
:103E300087E78093E50481E08093E6041092E7042D
:103E400083E090E00E94B201089581E78093E50449
:103E50000E945F1E8093E6041092E70483E090E0E6
:103E60000E94B2010895462F90E79093E50462E026
:103E70000E94921B8093E6041092E70483E090E096
:103E80000E94B2010895EF92FF920F931F93FC01DD
:103E90008081833701F1843748F48137C9F0823754
:103EA00008F06BC0803709F081C00DC0853709F478
:103EB0006CC0853708F45DC0863709F46AC087375F
:103EC00009F074C06BC0638182810E94331F79C086
:103ED0000E94251F76C000002581332744275527DF
:103EE000542F432F322F222786819927AA27BB27B9
:103EF000DC0199278827280F391F4A1F5B1F8481FF
:103F0000280F311D411D511D87819927AA27BB27E5
:103F1000B82FAA2799278827280F391F4A1F5B1F08
:103F2000E184FF2400271127102F0F2DFE2CEE24F3
:103F300082859927AA27BB27DC0199278827E80EC5
:103F4000F91E0A1F1B1F8085E80EF11C011D111DA3
:103F500083859927AA27BB27B82FAA2799278827BF
:103F6000E80EF91E0A1F1B1F638182810E94001F39
:103F700028C082810E94E41E24C0AF014C5F5F4FC5
:103F8000638182810E94F21E1CC082810E94D61E23
:103F900018C0828199270E94971E13C0AF014C5F01
:103FA0005F4F638182810E94161F0BC08093E504DE
:103FB00083E08093E6041092E70483E090E00E949F
:103FC000B2011F910F91FF90EF9008951F920F92F1
:103FD0000FB60F9211241F932F933F934F935F932C
:103FE0006F937F938F939F93AF93BF93EF93FF93C1
:103FF0001091ED000E94341E8F3F31F18295807F39
:104000008093ED000E94131C60936806709369060C
:1040100080936A0690936B068CE696E00E94001EE1
:104020000E94131C609368067093690680936A0669
:1040300090936B068091EE008F7D8093EE0083E07D
:104040000E94A91C1093ED00FF91EF91BF91AF91D9
:104050009F918F917F916F915F914F913F912F91A0
:104060001F910F900FBE0F901F901895DC0180E1FB
:10407000A030B80718F082E090E00895F999FECFDB
:104080009D0109C032BD21BD2F5F3F4FF89AE60F59
:10409000F71F80B58083822F8A1BE82FFF27E41744
:1040A000F50780F381E090E00895DC0180E1A03025
:1040B000B80718F082E090E00895F999FECF9D01CD
:1040C0000AC032BD21BD2F5F3F4FE60FF71F808131
:1040D00080BDFA9AF99A822F8A1BE82FFF27E417EE
:1040E000F50778F381E090E008950F931F938B011B
:1040F00021E82093E5040E9455208093E604109265
:10410000E7041F930F9384EF92E09F938F930E9495
:10411000FD1A83E090E00E94B2010F900F900F9083
:104120000F901F910F910895CF92DF92EF92FF921F
:104130000F931F937B0105EE14E020E82093E50424
:1041400022E0C22ED12CC00ED11EAB01B6010E94BE
:1041500036208093E60482E090E0E80EF91E0E0D12
:104160001F1DF8011082DF92CF9281E093E09F93B0
:104170008F930E94FD1AC70101960E94B2010F9011
:104180000F900F900F901F910F91FF90EF90DF9085
:10419000CF900895EF92FF920F931F93CF93DF93E9
:1041A000EC018B819927F82EEE248A81E80EF11C10
:1041B0008D819927182F00278C81080F111DFF92E0
:1041C000EF921F930F938BE093E09F938F930E9446
:1041D000FD1A88812DB73EB72A5F3F4F0FB6F8947E
:1041E0003EBF0FBE2DBF803819F0813869F405C07D
:1041F000B801C7010E94942012C02696A801BE01F2
:10420000C7010E9475200BC08093E50483E0809372
:10421000E6041092E70483E090E00E94B201DF918F
:10422000CF911F910F91FF90EF900895CF93DF935F
:10423000AC01029710F442E050E0A0917706B091F3
:104240007806FD01C0E0D0E020E030E020C08081B1
:1042500091818417950769F482819381209719F0E1
:104260009B838A8304C090937806809377069F018E
:1042700032C04817590738F42115310519F0821753
:10428000930708F49C01EF010280F381E02D309741
:10429000F1F62115310599F1C901841B950B04979D
:1042A00008F4A901E0E0F0E028C08D919C911197FD
:1042B00082179307F9F44817590781F4ED018A81B1
:1042C0009B81309719F09383828304C09093780682
:1042D000809377069D012E5F3F4F4CC0841B950B4A
:1042E000FD01E80FF91F4193519302978D939C9321
:1042F0009F0140C0FD01A281B3811097B1F680916A
:10430000750690917606892B41F480913203909145
:104310003303909376068093750620913403309191
:1043200035032115310549F48DB7282F33278091A6
:10433000300390913103281B390BA0917506B09181
:1043400076062A1B3B0B2417350790F0CA0102960C
:104350002817390768F09D012E5F3F4FC901840F70
:10436000951F90937606809375064D935C9302C0DB
:1043700020E030E0C901DF91CF910895CF93DF9322
:10438000009709F44EC0EC0122971B821A82A0917B
:104390007706B0917806109711F140E050E001C027
:1043A000DC01AC17BD0700F1BB83AA83FE0121919C
:1043B0003191E20FF31FEA17FB0771F48D919C9185
:1043C0001197280F391F2E5F3F4F39832883FD0136
:1043D000828193819B838A834115510559F4D0933F
:1043E0007806C09377061DC0FD0182819381AD01DF
:1043F0000097B1F6FA01D383C28321913191E20F84
:10440000F31FEC17FD0769F488819981280F391F84
:104410002E5F3F4FFA01318320838A819B819383F2
:104420008283DF91CF91089597FB092E07260AD04A
:1044300077FD04D00CD006D000201AF47095619559
:104440007F4F0895F6F7909581959F4F0895AA1B89
:10445000BB1B51E107C0AA1FBB1FA617B70710F06F
:10446000A61BB70B881F991F5A95A9F780959095A1
:08447000BC01CD010895FFCF4E
:10447800456D62656464656450726F6A65637473E0
:10448800004F63746F70757355534220496E74659D
:10449800726661636520436F6E766572746572201B
:1044A800616E6420492F4F20457874656E73696F7B
:1044B8006E003230303831313038006669727374CA
:1044C800207061636B6574206F662061206C6F6E6D
:1044D80067206D65737361676520286C656E677406
:1044E800683A202564290A006F63746F7075732019
:1044F8006C6F6E672072756E6E696E67206D65737E
:10450800736167650A006F63746F7075732E6C6FE3
:104518006E675F696E646578203C206F63746F70A6
:1045280075732E6C6F6E675F62797465730A006EBF
:104538006F74206C617374207061636B65743A20CA
:1045480064696666203E2036340A006C6173742004
:104558007061636B65740A007061727365722C20F8
:10456800636865636B3A2025582C20636F6D6D6115
:104578006E643A2025580A0063616C6C696E672086
:10458800696F5F7061727365720A0063616C6C6950
:104598006E67206164635F7061727365720A00639D
:1045A800616C6C696E67206932635F7061727365F4
:1045B800720A0063616C6C696E67207370695F7062
:1045C80061727365720A0063616C6C696E67207052
:1045D800776D5F7061727365720A0063616C6C69F4
:1045E8006E672063616E5F7061727365720A006343
:1045F800616C6C696E6720656570726F6D5F706164
:10460800727365720A00756E6B6E6F776E20636DDC
:10461800640A00726563656976696E6720636F6D09
:104628006D616E643A20255820286C656E67746841
:104638003A202575290A00676574206E6578740A22
:104648000067657420616E642065786563757465BC
:104658000A0009040000010203040506070001021C
:10466800030405067772697474656E3A2025730A27
:1046780000726561643A2025730A00656570726F7F
:104688006D5F7061727365723A206C656E677468ED
:104698003A2025752C20616464723A2025750A0039
:0646A8002000790600006D
:00000001FF
